:100000000C9472000C948D000C948D000C948D0057
:100010000C948D000C948D000C948D000C948D002C
:100020000C948D000C948D000C948D000C948D001C
:100030000C948D000C948D000C948D000C948D000C
:100040000C948D000C948D000C948D000C948D00FC
:100050000C948D000C948D000C948D000C948D00EC
:100060000C948D000C948D000C948D000C948D00DC
:100070000C948D000C948D000C948D000C948D00CC
:100080000C948D000C948D000C948D000C948D00BC
:100090000C948D000C948D000C948D000C948D00AC
:1000A0000C948D000C948D000C948D000C948D009C
:1000B0000C948D000C948D000C948D000C948D008C
:1000C0000C948D000C948D000C948D000C948D007C
:1000D0000C948D000C948D000C948D000C948D006C
:1000E0000C948D0011241FBECFEFD1E2DEBFCDBF37
:1000F00000E00CBF84B78093000214BE0FB6F894E2
:10010000A8958091600088618093600010926000E3
:100110000FBE0E94DD000C946E010C9400008093D1
:1001200008010895A8E0B1E08C938FEF80BBEBE06D
:10013000F1E080818D7F808361BB8081877F8083B8
:1001400085E08A95F1F700008081886080831C92A9
:1001500080818260808311BA0895A8E0B1E08C9319
:1001600010BA11BAEBE0F1E080818B7F808380814F
:10017000877F808385E08A95F1F700008FB19081B9
:10018000986090831C929081946090839FEF90BBC5
:1001900011BA95E09A95F1F70000089585E00E9464
:1001A000AD0080FF07C080E00E94AD00682F80E0B6
:1001B0000E94920090E080E00895F8948FEF80BB59
:1001C0008093070180930A0111BA109208011092DE
:1001D0000B0180910B01826080930B0180910B01D8
:1001E000846080930B0180910B01886080930B01E8
:1001F00080910B01806180930B0180910B018160E4
:1002000080930B018FE891E00197F1F700C00000A7
:1002100080910B018E7F80930B018FE99FE0019706
:10022000F1F700C0000063E883E00E94920063E001
:1002300080E00E94920060E081E00E94920063E012
:1002400083E00E94920069E480E00E9492008FE3C4
:100250009CE90197F1F700C000006EE480E00E9485
:1002600092008FE39CE90197F1F700C0000069E478
:1002700080E00E9492008FE39CE90197F1F700C0B3
:10028000000064E580E00E9492008FE39CE9019702
:10029000F1F700C000006DE080E00E9492008FE363
:1002A0009CE90197F1F700C000006AE080E00E943D
:1002B00092008FE39CE90197F1F700C00000789469
:1002C00088E19EE00FB6F894A895809360000FBE79
:1002D00090936000A8950E94CE00FCCFF894FFCFC9
:00000001FF
